:020000000528D1
:0800080013288501860183160F
:10001000F030860085019B0183128B018B158B17B5
:1000200007308600122806081A208500073086004F
:100030000B100900A0010130A2002208043C031C9F
:1000400043282208860000000000000000008030E5
:10005000A1000608A30010302102031C3D2823083C
:100060002105FF39003C031936284328A00A21083E
:10007000A400240C7F39A1002B282208A400240D01
:10008000FE39A2001D282008A4004F3E00300318AE
:10009000013E8A0024084E200800080082070A3426
:1000A00007340434013400340834053402340B348A
:1000B000093406340334FF3482072A3437343434A5
:1000C00031343034383435343234233439343634FE
:0400D0003334FF3492
:02400E002A3F47
:02401000FC3F73
:00000001FF
